:020000040000FA
:0408000002EF06F00D
:1008100003B20CEF05F0F2B427EF05F09EB02FEF16
:1008200005F0F2A817EF04F0F2B219EF04F0E0EFD0
:1008300005F0CD90F2929EA023EF04F00101463F17
:1008400023EF04F0472B81C185F182C186F183C17A
:1008500087F184C188F17DC181F17EC182F17FC1C0
:1008600083F180C184F179C17DF17AC17EF17BC1D0
:100870007FF17CC180F175C179F176C17AF177C1E0
:100880007BF178C17CF171C175F172C176F173C1F0
:1008900077F174C178F16DC171F16EC172F16FC100
:1008A00073F170C174F169C16DF16AC16EF16BC110
:1008B0006FF16CC170F1CECF69F1CFCF6AF146C153
:1008C0006BF147C16CF1CF6ACE6A0101466B476B91
:1008D0009E90CD800EBC0E8E0EBA72EF04F00E8A82
:1008E000E0EF05F00E8C0EBEAEEF04F069C16DF1C5
:1008F0006AC16EF16BC16FF16CC170F16DC171F1C4
:100900006EC172F16FC173F170C174F171C175F193
:1009100072C176F173C177F174C178F175C179F163
:1009200076C17AF177C17BF178C17CF179C17DF133
:100930007AC17EF17BC17FF17CC180F17DC181F103
:100940007EC182F17FC183F180C184F181C185F1D3
:1009500082C186F183C187F184C188F10101516BA5
:10096000526B536B546B695151276A5152236B512F
:1009700053236C5154236D5151276E5152236F51A3
:100980005323705154237151512772515223735183
:100990005323745154237551512776515223775163
:1009A000532378515423795151277A5152237B5143
:1009B00053237C5154237D5151277E5152237F5123
:1009C0005323805154238151512782515223835103
:1009D00053238451542385515127865152238751E3
:1009E000532388515423D8905433533352335133C3
:1009F000D8905433533352335133D8905433533304
:100A00005233513369C151F16AC152F16BC153F193
:100A10006CC154F1E0EF05F00392030103EE00F026
:100A200080517F0BE92604C0EFFF802B8151805D50
:100A3000700BD8A48B8200008051815D700BD8A40C
:100A40008B9281518019D8B40790E0EF05F0F294B1
:100A50000101383FE0EF05F0392BE0EF05F09E9003
:100A60000101463FE0EF05F0472BE0EF05F09E92D5
:100A7000C3CF48F1C4CF49F1C28207B462EF05F099
:100A80003AC13EF13BC13FF13CC140F13DC141F1B2
:100A900051C155F152C156F153C157F154C158F1EA
:100AA000010148514E2749514F23E86A50230D2E2A
:100AB00062EF05F04FC14AF150C14BF14E6B4F6BE5
:100AC000506B078E0201002FE0EF05F03C0E006F27
:100AD00001015D6773EF05F05E6773EF05F05F6717
:100AE00073EF05F0606777EF05F0A7EF05F061C1E0
:100AF00000F162C101F163C102F164C103F10101BE
:100B0000010E046F000E056F000E066F000E076FDA
:100B1000F7EC12F000C161F101C162F102C163F1B1
:100B200003C164F100679CEF05F001679CEF05F0DD
:100B300002679CEF05F00367A7EF05F05DC161F167
:100B40005EC162F15FC163F160C164F10E80D57E68
:100B5000D5BE34D0D6CF3AF1D7CF3BF138C13CF136
:100B6000E86AE8CF3DF10F80010147A7C4EF05F027
:100B70000E9A0E9C0E9E0101000E516F600E526F78
:100B80003D0E536F080E546F01013ABFD4EF05F0CC
:100B90003B67D4EF05F03C67D4EF05F03D67D4EF39
:100BA00005F0F288D9EF05F0F298516B526B536B58
:100BB000546BD76AD66A0101386B396BE0EF05F0E8
:100BC00002C0E0FF005001C0D8FF1000A6B2E6EF5F
:100BD00005F00CC0A9FF0BC0A8FFA69EA69CA6848A
:100BE000F29E550EA76EAA0EA76EA682F28EA6944E
:100BF000A6B2F8EF05F01200A96EA69EA69CA680EC
:100C0000A8501200076A0E6A0F6A0F010E0EC16E1D
:100C1000860EC06E030EC26E0F01080E8A6EF10EB4
:100C2000936E8B6A800E946EF18E0D6A01014E6B8D
:100C30004F6B506B4A6B4B6B0F01280ED56EF28ACF
:100C4000B00ECD6E9D800101516B526B536B546B96
:100C5000556B566B576B586B596B5A6B5B6B5C6B78
:100C60000E9A0E9C0E9EFF0ECB6E200EBB6E0C0ECF
:100C7000BA6E760ECA6E160EFCEC05F0E8CF00F1E7
:100C8000170EFCEC05F0E8CF01F1180EFCEC05F0B6
:100C9000E8CF02F1190EFCEC05F0E8CF03F10101F9
:100CA00003AF6DEF06F0EEEC13F0160E0C6E00C104
:100CB0000BF0E6EC05F0170E0C6E01C10BF0E6EC44
:100CC00005F0180E0C6E02C10BF0E6EC05F0190EE3
:100CD0000C6E03C10BF0E6EC05F000C15DF101C143
:100CE0005EF102C15FF103C160F100C161F101C1B8
:100CF00062F102C163F103C164F11A0EFCEC05F06C
:100D0000E8CF00F11B0EFCEC05F0E8CF01F11C0E62
:100D1000FCEC05F0E8CF02F11D0EFCEC05F0E8CF8D
:100D200003F1010103AFC3EF06F0EEEC13F01A0E6E
:100D30000C6E00C10BF0E6EC05F01B0E0C6E01C151
:100D40000BF0E6EC05F01C0E0C6E02C10BF0E6ECAD
:100D500005F01D0E0C6E03C10BF0E6EC05F01A0E4B
:100D6000FCEC05F0E8CF00F11B0EFCEC05F0E8CF41
:100D700001F11C0EFCEC05F0E8CF02F11D0EFCECBD
:100D800005F0E8CF03F100C165F101C166F102C1D0
:100D900067F103C168F1240EAC6E900EAB6E240EA9
:100DA000AC6E080EB86E000EB06E1F0EAF6E040172
:100DB000806B816B0F01900EAB6E0F019D8A03015A
:100DC000806B816BA26B8B9207900001F28EF28C8C
:100DD00007B0BBEF10F00EB0F9EF0BF0030180513C
:100DE00081197F0BD8B4BBEF10F013EE00F08151E6
:100DF0007F0BE126812BE7CFE8FFE00BD8B4BBEFF8
:100E000010F023EE82F0A2511F0BD926E7CFDFFFAF
:100E1000A22BDF50780AD8A4BBEF10F0078061C185
:100E200000F162C101F163C102F164C103F101018A
:100E3000040E046F000E056F000E066F000E076FA4
:100E4000F7EC12F000AF2EEF07F00101030E616F17
:100E5000000E626F000E636F000E646F030182511B
:100E6000720AD8B4F9EF0BF08251520AD8B4F9EFF4
:100E70000BF08251630AD8B477EF0DF08251690A02
:100E8000D8B4FEEF08F082517A0AD8B411EF0AF014
:100E90008251490AD8B49DEF08F08251500AD8B463
:100EA000BBEF07F08251700AD8B4FEEF07F0825111
:100EB000540AD8B429EF08F08251740AD8B46FEFFD
:100EC00008F08251730AD8B429EF0BF08251530A0B
:100ED000D8B48EEF0BF08251760AD8B48AEF07F0BF
:100EE0008251560AD8B4B9EF07F0ACEF0DF0040107
:100EF00014EE00F080517F0BE12682C4E7FF802BC7
:100F000012000D0E826F77EC07F00A0E826F77ECFD
:100F100007F012002FEC14F083C324F184C325F1F1
:100F200085C326F186C327F101013CEC14F0B3EC34
:100F300013F000C10CF101C10DF102C10EF103C1AA
:100F40000FF1D8900333023301330033D8900333C9
:100F50000233013300330C470C470C470C47300E6B
:100F60000C170C0E0C1300C1BBFF0CC1BAFFACEF89
:100F70000DF0ACEF0DF083C31EF184C31FF185C3E8
:100F800020F186C321F187C322F188C323F189C3ED
:100F900024F18AC325F18BC326F18CC327F101010B
:100FA0003CEC14F0B3EC13F0160E0C6E00C10BF019
:100FB000E6EC05F0170E0C6E01C10BF0E6EC05F047
:100FC000180E0C6E02C10BF0E6EC05F0190E0C6E5B
:100FD00003C10BF0E6EC05F000C15DF101C15EF16B
:100FE00002C15FF103C160F100C161F101C162F1B1
:100FF00002C163F103C164F19DEF08F083C31EF1E8
:1010000084C31FF185C320F186C321F187C322F178
:1010100088C323F189C324F18AC325F18BC326F148
:101020008CC327F101013CEC14F0B3EC13F000C1C8
:101030005DF101C15EF102C15FF103C160F100C168
:1010400061F101C162F102C163F103C164F19DEF7D
:1010500008F083C31EF184C31FF185C320F186C34A
:1010600021F187C322F188C323F189C324F18AC304
:1010700025F18CC326F18DC327F101013CEC14F05E
:10108000B3EC13F00101000E046F000E056F010EAA
:10109000066F000E076F06EC13F01A0E0C6E00C1FF
:1010A0000BF0E6EC05F01B0E0C6E01C10BF0E6EC4C
:1010B00005F01C0E0C6E02C10BF0E6EC05F01D0EE7
:1010C0000C6E03C10BF0E6EC05F000C165F101C147
:1010D00066F102C167F103C168F19DEF08F083C3B7
:1010E0001EF184C31FF185C320F186C321F187C39C
:1010F00022F188C323F189C324F18AC325F18CC36B
:1011000026F18DC327F101013CEC14F0B3EC13F090
:101110000101000E046F000E056F010E066F000E38
:10112000076F06EC13F000C165F101C166F102C161
:1011300067F103C168F19DEF08F0160EFCEC05F0B5
:10114000E8CF00F1170EFCEC05F0E8CF01F1180E26
:10115000FCEC05F0E8CF02F1190EFCEC05F0E8CF4D
:1011600003F191EC13F0BDEC11F00401730E826FEA
:1011700077EC07F004012C0E826F77EC07F05DC16D
:1011800000F15EC101F15FC102F160C103F191ECB8
:1011900013F0BDEC11F00401730E826F77EC07F0D1
:1011A00004012C0E826F77EC07F01A0EFCEC05F0B0
:1011B000E8CF00F11B0EFCEC05F0E8CF01F11C0EAE
:1011C000FCEC05F0E8CF02F11D0EFCEC05F0E8CFD9
:1011D00003F1C7EC0DF004012C0E826F77EC07F0E1
:1011E00065C100F166C101F167C102F168C103F197
:1011F000C7EC0DF081EC07F0ACEF0DF00401690EC7
:10120000826F77EC07F004012C0E826F77EC07F009
:101210000101040E006F000E016F000E026F000E40
:10122000036F91EC13F020C182F40401300E822789
:1012300077EC07F021C182F40401300E822777ECAD
:1012400007F022C182F40401300E822777EC07F008
:1012500023C182F40401300E822777EC07F024C109
:1012600082F40401300E822777EC07F025C182F466
:101270000401300E822777EC07F026C182F40401C6
:10128000300E822777EC07F027C182F40401300E7C
:10129000822777EC07F004012C0E826F77EC07F0C1
:1012A0000101090E006F000E016F000E026F000EAB
:1012B000036F91EC13F020C182F40401300E8227F9
:1012C00077EC07F021C182F40401300E822777EC1D
:1012D00007F022C182F40401300E822777EC07F078
:1012E00023C182F40401300E822777EC07F024C179
:1012F00082F40401300E822777EC07F025C182F4D6
:101300000401300E822777EC07F026C182F4040135
:10131000300E822777EC07F027C182F40401300EEB
:10132000822777EC07F004012C0E826F77EC07F030
:101330000101130E006F000E016F000E026F000E10
:10134000036F91EC13F020C182F40401300E822768
:1013500077EC07F021C182F40401300E822777EC8C
:1013600007F022C182F40401300E822777EC07F0E7
:1013700023C182F40401300E822777EC07F024C1E8
:1013800082F40401300E822777EC07F025C182F445
:101390000401300E822777EC07F026C182F40401A5
:1013A000300E822777EC07F027C182F40401300E5B
:1013B000822777EC07F004012C0E826F77EC07F0A0
:1013C000200EF86EF76AF66A04010900F5CF82F480
:1013D00077EC07F00900F5CF82F477EC07F009000D
:1013E000F5CF82F477EC07F00900F5CF82F477ECC3
:1013F00007F00900F5CF82F477EC07F00900F5CF8C
:1014000082F477EC07F00900F5CF82F477EC07F06F
:101410000900F5CF82F477EC07F081EC07F0ACEF30
:101420000DF08351630AD8A4ACEF0DF08451610A2A
:10143000D8A4ACEF0DF085516C0AD8A4ACEF0DF038
:101440008651410A42E08651440A1BE08651420A15
:10145000D8B478EF0AF08651350AD8B436EF0FF0D9
:101460008651360AD8B48BEF0FF08651370AD8B4BC
:10147000F4EF0FF08651380AD8B452EF10F0ACEF09
:101480000DF00798079A04017A0E826F77EC07F047
:101490000401780E826F77EC07F00401640E826F0E
:1014A00077EC07F081A85CEF0AF00401550E826F1B
:1014B00077EC07F061EF0AF004014C0E826F77ECD5
:1014C00007F081EC07F0ACEF0DF00788079A0401F4
:1014D0007A0E826F77EC07F00401410E826F77EC91
:1014E00007F00401610E826F77EC07F052EF0AF00B
:1014F0000798078A04017A0E826F77EC07F00401DF
:10150000420E826F77EC07F00401610E826F77EC78
:1015100007F052EF0AF00101620E046F010E056F31
:10152000000E066F000E076F59C100F15AC101F19C
:101530005BC102F15CC103F1F7EC12F003BFE8EF0D
:101540000AF00E0EFCEC05F0E8CF0CF10F0EFCECEF
:1015500005F0E8CF0DF1100EFCEC05F0E8CF0EF130
:10156000110EFCEC05F0E8CF0FF140EC12F059C180
:1015700004F15AC105F15BC106F15CC107F1F7EC5A
:1015800012F0078204EC12F040EC12F0079204EC27
:1015900012F059C100F15AC101F15BC102F15CC105
:1015A00003F1079204EC12F0CC0E046FE00E056F0D
:1015B000870E066F050E076FF7EC12F000C10CF1F5
:1015C00001C10DF102C10EF103C10FF120EF0BF0CB
:1015D0000101800E006F1A0E016F060E026F000EE1
:1015E000036F42C104F143C105F144C106F145C195
:1015F00007F1F7EC12F003AF01EF0BF0EEEC13F094
:1016000012000E0EFCEC05F0E8CF0CF10F0EFCEC16
:1016100005F0E8CF0DF1100EFCEC05F0E8CF0EF16F
:10162000110EFCEC05F0E8CF0FF142C100F143C10F
:1016300001F144C102F145C103F1078204EC12F04B
:101640000CC100F10DC101F10EC102F10FC103F196
:1016500012000401730E826F77EC07F004012C0E68
:10166000826F77EC07F0078455C159F156C15AF1E2
:1016700057C15BF158C15CF13EC142F13FC143F13A
:1016800040C144F141C145F14AC14CF14BC14DF15A
:1016900007944FEC0BF081EC07F0ACEF0DF059C163
:1016A00000F15AC101F15BC102F15CC103F101011A
:1016B00091EC13F0BDEC11F00401630E826F77EC36
:1016C00007F004012C0E826F77EC07F042C100F1A5
:1016D00043C101F144C102F145C103F1010191ECA3
:1016E00013F0BDEC11F00401660E826F77EC07F089
:1016F00004012C0E826F77EC07F0EEEC13F04CC176
:1017000000F14DC101F1010191EC13F0BDEC11F0BC
:101710000401740E826F77EC07F012000F8204014F
:10172000530E826F77EC07F004012C0E826F77EC7A
:1017300007F083C31EF184C31FF185C320F186C364
:1017400021F187C322F188C323F189C324F18AC31D
:1017500025F18BC326F18CC327F101013CEC14F079
:10176000B3EC13F000C159F101C15AF102C15BF1B0
:1017700003C15CF18EC31EF18FC31FF190C320F132
:1017800091C321F192C322F193C323F194C324F1B5
:1017900095C325F196C326F197C327F101013CECCF
:1017A00014F0B3EC13F000C142F101C143F102C1E6
:1017B00044F103C145F12FEC14F099C323F19AC30E
:1017C00024F19BC325F19CC326F19DC327F10101A0
:1017D0003CEC14F0B3EC13F000C14CF101C14DF13D
:1017E0004FEC0BF004012C0E826F77EC07F000EF4A
:1017F0000CF08251520A03E10E8200EF0CF00E92BF
:1018000007840FB218EF0CF055C159F156C15AF1C7
:1018100057C15BF158C15CF13EC142F13FC143F198
:1018200040C144F141C145F14AC14CF14BC14DF1B8
:1018300007940EA03AEF0CF00101656727EF0CF05A
:10184000666727EF0CF0676727EF0CF068672BEFF0
:101850000CF03AEF0CF08BEC0AF065C104F166C1B4
:1018600005F167C106F168C107F1F7EC12F003BF9B
:1018700074EF0DF08BEC0AF00101000E046F000E06
:10188000056F010E066F000E076F25EC13F00401C3
:10189000720E826F77EC07F004012C0E826F77ECEA
:1018A00007F091EC13F01D675BEF0CF00401200EC4
:1018B000826F5EEF0CF004012D0E826F77EC07F063
:1018C00024C182F40401300E822777EC07F025C191
:1018D00082F40401300E822777EC07F004012E0E0B
:1018E000826F77EC07F026C182F40401300E822764
:1018F00077EC07F027C182F40401300E822777ECE1
:1019000007F004016D0E826F77EC07F004012C0ED6
:10191000826F77EC07F042C100F143C101F144C18D
:1019200002F145C103F1010191EC13F0BDEC11F09E
:101930000401480E826F77EC07F004017A0E826F83
:1019400077EC07F004012C0E826F77EC07F059C199
:1019500000F15AC101F15BC102F15CC103F1010167
:1019600091EC13F0BDEC11F00401630E826F77EC83
:1019700007F004012C0E826F77EC07F059C100F1DB
:101980005AC101F15BC102F15CC103F101010A0E10
:10199000046F000E056F000E066F000E076F06EC59
:1019A00013F0000E046F120E056F000E066F000E8E
:1019B000076F25EC13F091EC13F01EC182F40401C3
:1019C000300E822777EC07F01FC182F40401300E3D
:1019D000822777EC07F020C182F40401300E8227C1
:1019E00077EC07F021C182F40401300E822777ECF6
:1019F00007F022C182F40401300E822777EC07F051
:101A000023C182F40401300E822777EC07F024C151
:101A100082F40401300E822777EC07F004012E0EC9
:101A2000826F77EC07F025C182F40401300E822723
:101A300077EC07F026C182F40401300E822777ECA0
:101A400007F027C182F40401300E822777EC07F0FB
:101A50000401730E826F77EC07F004012C0E826F85
:101A600077EC07F0EEEC13F04CC100F14DC101F141
:101A7000D6EC0EF00EB240EF0DF00EA072EF0DF0AE
:101A800004012C0E826F77EC07F0200EF86EF76AD7
:101A9000F66A04010900F5CF82F477EC07F009003B
:101AA000F5CF82F477EC07F00900F5CF82F477ECFC
:101AB00007F00900F5CF82F477EC07F00900F5CFC5
:101AC00082F477EC07F00900F5CF82F477EC07F0A9
:101AD0000900F5CF82F477EC07F00900F5CF82F426
:101AE00077EC07F081EC07F00E90ACEF0DF00401FD
:101AF000630E826F77EC07F004012C0E826F77EC97
:101B000007F0B2EC0DF004012C0E826F77EC07F0B9
:101B100025EC0EF004012C0E826F77EC07F0A1EC9F
:101B20000EF004012C0E826F77EC07F00101F80E25
:101B3000006FCD0E016F660E026F030E036FC7ECD0
:101B40000DF004012C0E826F77EC07F0B7EC0EF06D
:101B500081EC07F0ACEF0DF00301A26B07900F9240
:101B6000BBEF10F0D8900E0EFCEC05F0E8CF00F1C2
:101B70000F0EFCEC05F0E8CF01F1100EFCEC05F0C7
:101B8000E8CF02F1110EFCEC05F0E8CF03F1010102
:101B9000000E046F000E056F010E066F000E076F3A
:101BA00025EC13F091EC13F01EC182F40401300E09
:101BB000822777EC07F01FC182F40401300E8227E0
:101BC00077EC07F020C182F40401300E822777EC15
:101BD00007F021C182F40401300E822777EC07F070
:101BE00022C182F40401300E822777EC07F023C172
:101BF00082F40401300E822777EC07F024C182F4CE
:101C00000401300E822777EC07F025C182F404012D
:101C1000300E822777EC07F004012E0E826F77ECEE
:101C200007F026C182F40401300E822777EC07F01A
:101C300027C182F40401300E822777EC07F00401FB
:101C40006D0E826F77EC07F01200120EFCEC05F0BF
:101C5000E8CF00F1130EFCEC05F0E8CF01F1140E13
:101C6000FCEC05F0E8CF02F1150EFCEC05F0E8CF36
:101C700003F101010A0E046F000E056F000E066FDE
:101C8000000E076F06EC13F0000E046F120E056FC6
:101C9000000E066F000E076F25EC13F091EC13F0A9
:101CA0001EC182F40401300E822777EC07F01FC1B9
:101CB00082F40401300E822777EC07F020C182F411
:101CC0000401300E822777EC07F021C182F4040171
:101CD000300E822777EC07F022C182F40401300E27
:101CE000822777EC07F023C182F40401300E8227AB
:101CF00077EC07F024C182F40401300E822777ECE0
:101D000007F004012E0E826F77EC07F025C182F4F4
:101D10000401300E822777EC07F026C182F404011B
:101D2000300E822777EC07F027C182F40401300ED1
:101D3000822777EC07F00401730E826F77EC07F0CF
:101D400012000A0EFCEC05F0E8CF00F10B0EFCECE3
:101D500005F0E8CF01F10C0EFCEC05F0E8CF02F144
:101D60000D0EFCEC05F0E8CF03F1D6EF0EF0060EF9
:101D7000FCEC05F0E8CF00F1070EFCEC05F0E8CF35
:101D800001F1080EFCEC05F0E8CF02F1090EFCECC5
:101D900005F0E8CF03F1D6EF0EF00101EEEC13F001
:101DA00007844AC100F14BC101F107940101E80E1B
:101DB000046F800E056F000E066F000E076F06ECB5
:101DC00013F0000E046F040E056F000E066F000E78
:101DD000076F25EC13F0880E046F130E056F000ECD
:101DE000066F000E076FF7EC12F00A0E046F000E7C
:101DF000056F000E066F000E076F25EC13F091ECD7
:101E000013F001011D670AEF0FF00401200E826F2D
:101E10000DEF0FF004012D0E826F77EC07F024C157
:101E200082F40401300E822777EC07F025C182F49A
:101E30000401300E822777EC07F026C182F40401FA
:101E4000300E822777EC07F004012E0E826F77ECBC
:101E500007F027C182F40401300E822777EC07F0E7
:101E60000401430E826F77EC07F0120087C31EF166
:101E700088C31FF189C320F18AC321F18BC322F1EA
:101E80008CC323F18DC324F18EC325F190C326F1B9
:101E900091C327F101011D6B3CEC14F0B3EC13F07E
:101EA0000101000E046F000E056F010E066F000E9B
:101EB000076F06EC13F00E0E0C6E00C10BF0E6EC93
:101EC00005F00F0E0C6E01C10BF0E6EC05F0100EE4
:101ED0000C6E02C10BF0E6EC05F0110E0C6E03C1A6
:101EE0000BF0E6EC05F004017A0E826F77EC07F058
:101EF00004012C0E826F77EC07F00401350E826F1F
:101F000077EC07F004012C0E826F77EC07F0B2EC4F
:101F10000DF061EF0AF087C31EF188C31FF189C37A
:101F200020F18AC321F18BC322F18CC323F18DC32D
:101F300024F18EC325F190C326F191C327F101014D
:101F40001D6B3CEC14F0B3EC13F0880E046F130E11
:101F5000056F000E066F000E076FFBEC12F0000E0F
:101F6000046F040E056F000E066F000E076F06EC7F
:101F700013F00101E80E046F800E056F000E066F6E
:101F8000000E076F25EC13F00A0E0C6E00C10BF06B
:101F9000E6EC05F00B0E0C6E01C10BF0E6EC05F063
:101FA0000C0E0C6E02C10BF0E6EC05F00D0E0C6E83
:101FB00003C10BF0E6EC05F004017A0E826F77ECBA
:101FC00007F004012C0E826F77EC07F00401360E47
:101FD000826F77EC07F004012C0E826F77EC07F02C
:101FE000A1EC0EF061EF0AF087C31EF188C31FF168
:101FF00089C320F18AC321F18BC322F18CC323F161
:102000008DC324F18FC325F190C326F191C327F12D
:1020100001013CEC14F0B3EC13F0000E046F120E4F
:10202000056F000E066F000E076F06EC13F001013E
:102030000A0E046F000E056F000E066F000E076F8C
:1020400025EC13F0120E0C6E00C10BF0E6EC05F05F
:10205000130E0C6E01C10BF0E6EC05F0140E0C6EC5
:1020600002C10BF0E6EC05F0150E0C6E03C10BF08F
:10207000E6EC05F004017A0E826F77EC07F00401BC
:102080002C0E826F77EC07F00401370E826F77EC2D
:1020900007F004012C0E826F77EC07F025EC0EF0B0
:1020A00061EF0AF087C31EF188C31FF189C320F1D5
:1020B0008AC321F18BC322F18CC323F18DC324F198
:1020C0008EC325F190C326F191C327F101011D6B49
:1020D0003CEC14F0B3EC13F0880E046F130E056F94
:1020E000000E066F000E076FFBEC12F0000E046F7F
:1020F000040E056F000E066F000E076F06EC13F05E
:102100000101E80E046F800E056F000E066F000ED1
:10211000076F25EC13F0060E0C6E00C10BF0E6EC19
:1021200005F0070E0C6E01C10BF0E6EC05F0080E91
:102130000C6E02C10BF0E6EC05F0090E0C6E03C14B
:102140000BF0E6EC05F004017A0E826F77EC07F0F5
:1021500004012C0E826F77EC07F00401380E826FB9
:1021600077EC07F004012C0E826F77EC07F0B7ECE8
:102170000EF061EF0AF081A879EF11F007A832EFB5
:1021800011F00101800E006F1A0E016F060E026F32
:10219000000E036F3EC104F13FC105F140C106F1DD
:1021A00041C107F1F7EC12F003BF79EF11F0B7EC82
:1021B00011F03EC100F13FC101F140C102F141C146
:1021C00003F1078204EC12F00CC104F10DC105F11A
:1021D0000EC106F10FC107F1F80E006FCD0E016FB1
:1021E000660E026F030E036FF7EC12F00E0E0C6E0C
:1021F00000C10BF0E6EC05F00F0E0C6E01C10BF008
:10220000E6EC05F0100E0C6E02C10BF0E6EC05F0EA
:10221000110E0C6E03C10BF0E6EC05F00784010112
:10222000EEEC13F04AC100F14BC101F107940A0E24
:102230000C6E00C10BF0E6EC05F00B0E0C6E01C14C
:102240000BF0E6EC05F00C0E0C6E02C10BF0E6ECA8
:1022500005F00D0E0C6E03C10BF0E6EC05F00798CF
:1022600079EF11F007AA79EF11F007840101EEEC84
:1022700013F04AC100F14BC101F10794060E0C6E38
:1022800000C10BF0E6EC05F0070E0C6E01C10BF07F
:10229000E6EC05F0080E0C6E02C10BF0E6EC05F062
:1022A000090E0C6E03C10BF0E6EC05F0078455C176
:1022B00000F156C101F157C102F158C103F1079471
:1022C000120E0C6E00C10BF0E6EC05F0130E0C6E56
:1022D00001C10BF0E6EC05F0140E0C6E02C10BF020
:1022E000E6EC05F0150E0C6E03C10BF0E6EC05F004
:1022F000079A0401805181197F0B0BE09EA809D039
:1023000014EE00F081517F0BE126E750812B0F0185
:10231000AD6EE8EF06F00CC100F10DC101F10EC188
:1023200002F10FC103F1000E046F000E056F010EE4
:10233000066F000E076F25EC13F01DA1B6EF11F02C
:102340001451D8B4B6EF11F00CC100F10DC101F178
:102350000EC102F10FC103F1000E046F000E056FF4
:102360000A0E066F000E076F25EC13F01200010134
:102370000C6B0D6B0E6B0F6B12001EC182F404010F
:10238000300E822777EC07F01FC182F40401300E73
:10239000822777EC07F020C182F40401300E8227F7
:1023A00077EC07F021C182F40401300E822777EC2C
:1023B00007F022C182F40401300E822777EC07F087
:1023C00023C182F40401300E822777EC07F024C188
:1023D00082F40401300E822777EC07F025C182F4E5
:1023E0000401300E822777EC07F026C182F4040145
:1023F000300E822777EC07F027C182F40401300EFB
:10240000822777EC07F012000101005305E1015328
:1024100003E1025301E1002BC7EC12F0EEEC13F0E4
:102420002C51006F2D51016F420E046F4B0E056F42
:10243000000E066F000E076F06EC13F000C104F1EA
:1024400001C105F102C106F103C107F10CC100F1A0
:102450000DC101F10EC102F10FC103F107B235EF59
:1024600012F0FBEC12F037EF12F0F7EC12F000C1B3
:102470000CF101C10DF102C10EF103C10FF1120007
:10248000EEEC13F04CC100F14DC101F1060EFCEC75
:1024900005F0E8CF04F1070EFCEC05F0E8CF05F1FC
:1024A000080EFCEC05F0E8CF06F1090EFCEC05F097
:1024B000E8CF07F1F7EC12F000C118F101C119F1F2
:1024C00002C11AF103C11BF1290E046F000E056F42
:1024D000000E066F000E076F06EC13F0EE0E046F91
:1024E000430E056F000E066F000E076FFBEC12F037
:1024F00018C104F119C105F11AC106F11BC107F198
:1025000006EC13F000C110F101C111F102C112F18A
:1025100003C113F1120EFCEC05F0E8CF04F1130E29
:10252000FCEC05F0E8CF05F1140EFCEC05F0E8CF6B
:1025300006F1150EFCEC05F0E8CF07F10D0E006F6B
:10254000000E016F000E026F000E036F06EC13F019
:10255000180E046F000E056F000E066F000E076F59
:1025600025EC13F010C104F111C105F112C106F1FF
:1025700013C107F1FBEC12F06A0E046F2A0E056F0F
:10258000000E066F000E076FF7EC12F01200BF0E80
:10259000FA6E200E2D6F2C6BD89000370137023762
:1025A0000337D8B0D8EF12F02D2FCDEF12F02C0753
:1025B0002D070353D8B412000331070B8009326F83
:1025C00003390F0B010F2C6F80EC5FF0336F2C057C
:1025D00080EC5FF0335D335F2C6B3233D8B02C2747
:1025E0002C3332A9EDEF12F033512C27120013ECEB
:1025F00014F0D8B0120003510719286FD6EC13F06D
:10260000D8900751031928AF800F1200286BFAECFD
:1026100013F0D8A010EC14F0D8B01200E5EC13F0D1
:10262000EEEC13F01F0E296F26EC14F00B35D8B02A
:10263000D6EC13F0D8A00335D8B01200292F14EF30
:1026400013F028B1FDEC13F01200286B04510511B2
:10265000061107110008D8A0FAEC13F0D8A010EC6E
:1026600014F0D8B01200086B096B0A6B0B6B26ECE8
:1026700014F01F0E296F26EC14F007510B5DD8A43F
:102680004EEF13F006510A5DD8A44EEF13F005513A
:10269000095DD8A44EEF13F00451085DD8A061EF96
:1026A00013F00451085F0551D8A0053D095F06519C
:1026B000D8A0063D0A5F0751D8A0073D0B5FD89010
:1026C0000081292F3BEF13F028B1FDEC13F0286BAC
:1026D000FAEC13F0D8902AEC14F007510B5DD8A453
:1026E0007EEF13F006510A5DD8A47EEF13F005517A
:1026F000095DD8A47EEF13F00451085DD8A08DEFDA
:1027000013F0003F8DEF13F0013F8DEF13F0023F08
:102710008DEF13F0032BD8B4120028B1FDEC13F0A9
:1027200012000101286BFAEC13F0D8B012002FEC64
:1027300014F0200E296F003701370237033711EEEE
:1027400027F00A0E2A6FE7360A0EE75CD8B0E76E6C
:10275000E5522A2FA3EF13F0292F9BEF13F028B196
:102760001D81D890120001010A0E286F200E296FDA
:1027700011EE1DF028512A6F0A0ED890E652D8B0FB
:10278000E726E7322A2FBEEF13F00333023301337B
:102790000033292FB8EF13F0E750FF0FD8A003350F
:1027A000D8B012001DB1FDEC13F012000451002747
:1027B0000551D8B0053D01270651D8B0063D022786
:1027C0000751D8B0073D032712000051086F01518F
:1027D000096F02510A6F03510B6F12000101006B68
:1027E000016B026B036B12000101046B056B066B3E
:1027F000076B12000335D8A012000351800B001F95
:10280000011F021F031F003F0DEF14F0013F0DEFEA
:1028100014F0023F0DEF14F0032B282B03251200B8
:102820000735D8A012000751800B041F051F061F93
:10283000071F043F23EF14F0053F23EF14F0063F7A
:1028400023EF14F0072B282B072512000037013740
:1028500002370337083709370A370B3712000101EF
:102860001D6B1E6B1F6B206B216B226B236B246B0C
:10287000256B266B276B12001E510F0B1E6F1F510D
:102880000F0B1F6F20510F0B206F21510F0B216F6A
:1028900022510F0B226F23510F0B236F24510F0B6B
:1028A000246F25510F0B256F26510F0B266F2751D3
:0628B0000F0B276F120060
:10BF0000E844F926000C160C2B0C3F0C520C640C68
:10BF1000760C860C960CA50CB30CC10CCF0CDC0C6B
:06BF2000E80CF40C000C1B
:00000001FF
